:020000020000FC
:020000000DC031
:040010002AC124C11C
:100018001895189504E00EBF0FE50DBF02E003BF69
:1000280000E00DBD00E00CBD00E00BBD00E20ABD24
:1000380000E00FBD0BE00EBDA29ABA9ABB9AA59A32
:10004800B99ABC9AA09AA19AA39AA49A88988998CE
:100058008A988B988C98BE98BF988D988E988E9811
:10006800909A919A929A939A949AC69AC79A959ABC
:10007800969A969AB898C09ABD98C59A24E030E0A6
:1000880041E011D183D070E080E090E050E0AA24F4
:10009800D7D061606D7F6B7F789470E0B09B7160A2
:1000A800B59B7260B09B7160B59B7260703089F4CB
:1000B80090E080E05F3F61F053955F3F49F461FF56
:1000C80004C00FD16D7FAA2455D162FF01C06E7F95
:1000D8002DC060FD04C0616050E0872F27C07330D9
:1000E80051F462FF04C06B7F50D165D11EC06460BB
:1000F8004CD156D11AC050E09395903211F49FE13B
:1001080080E0803099F4713039F4F8941FD02CD005
:100118007894626081E009C0723041F4F89408D0A4
:1001280023D07894626082E000C030D0FBD0B5CF95
:1001380001E0400F4A3049F440E0300F3A3029F4EA
:1001480030E0200F2A3009F420E0089501E0401B38
:100158004F3F49F449E0301B3F3F29F439E0201B69
:100168002F3F09F429E00895253031F4313021F486
:10017800433059F442E009C0293039F4393029F4C0
:10018800493019F420E030E040E00895A0E0B0E004
:1001980004E6029FA00DB11D0AE0039FA00DB11D4A
:1001A800A40F0027B01FA5FBB2F9A6FBB3F9A7FB64
:1001B800A5F9B0FBA6F9B1FBA7F90A2F02BB0A2FD4
:1001C80001BBB2FFC698B2FDC69AB2FFBE98B2FD97
:1001D800BE9AB3FFC798B3FDC79AB3FFBF98B3FDE4
:1001E800BF9A0895A095B0950895F3E0EEEFE00F5B
:1001F8000027F01F04910895079510F0AD9A01C0EB
:10020800AD98079510F0C19A01C0C198079510F0F4
:10021800C49A01C0C498079510F0A89A01C0A8987C
:10022800079510F0A99A01C0A998079510F0AB9A04
:1002380001C0AB98079510F0AC9A01C0AC9808952E
:1002480001E109BF00E00BBF089500E009BF00E825
:100258000BBF0895CFB60F930F91CFBE1895CFB6A9
:100268000F939394AA98C298C39860FF19C0092D58
:10027800013029F4022FB9DFBFDFAA9A11C0092D76
:10028800023029F4032FB1DFB7DFC29A09C0092D64
:10029800033031F4042FA9DFAFDFC39A00E0902EBA
:1002A8000F91CFBE189534D000E00FBB00E00EBB15
:1002B80036D0063028F000E0202F302F402F089548
:1002C800202F26D000E00FBB01E00EBB28D0302F36
:1002D8001FD000E00FBB02E00EBB21D0402F18D08A
:1002E800089516D000E00FBB00E00EBB022F13D01C
:1002F8000FD000E00FBB01E00EBB032F0CD008D0DD
:1003080000E00FBB02E00EBB042F05D001D008951A
:10031800E199FECF08950DBBE29AE19A0895E09A1B
:100328000DB3089500E210E01A95F1F70A95E1F788
:10033800089503D00A95E9F708950F930AE00DD0C0
:100348000A950000E1F70F9108950F9301E005D099
:100358000A950000E1F70F9108950F9305E10A95BA
:100368000000E9F700000F9108950FEFE2DF0FEFAB
:10037800E0DF08952F933F934F9321E132E140E16D
:10038800F4DF4F913F912F9108952F933F934F930F
:100398002AE03BE04CE0E9DF4F913F912F9108952F
:1003A8002F933F934F932EE030E140E1DEDF4F91F2
:1003B8003F912F9108952F933F934F932DE03EE067
:1003C8004FE0D3DF4F913F912F9108952863292063
:1003D800576F6C6667616E672044756E637A6577E0
:1003E800736B69207777772E6D6964692D72616BFD
:1003F8006574652E64653F065B4F666D7D077F6F8C
:0A04080038795E005C54716D7700D6
:00000001FF
